:020000040800F2
:1000000000090020E9040008E1140008E5140008D4
:1000100039150008E51400080D150008EB04000868
:10002000EB040008EB040008EB040008A537000807
:10003000EB040008EB040008EB040008493C00084E
:10004000EB040008EB040008EB040008EB040008D4
:10005000EB040008EB0400082D3A0008593A0008A8
:10006000853A0008B13A0008DD3A0008EB040008C0
:10007000EB040008EB040008EB040008EB040008A4
:10008000EB040008EB040008EB040008512600080C
:10009000BD2600081127000865270008093B000855
:1000A000EB040008EB040008EB040008EB04000874
:1000B000EB040008EB040008EB040008EB04000864
:1000C000EB040008EB040008EB040008EB04000854
:1000D000EB040008EB040008212B0008352B000876
:1000E000713B0008EB040008EB040008EB04000877
:1000F000EB040008EB040008EB040008EB04000824
:10010000EB040008EB040008EB040008EB04000813
:10011000EB040008EB040008EB040008EB04000803
:10012000EB040008EB040008EB040008EB040008F3
:10013000EB040008EB040008EB040008EB040008E3
:10014000EB040008EB040008EB040008EB040008D3
:10015000EB040008EB040008EB040008EB040008C3
:10016000EB040008EB040008EB040008EB040008B3
:10017000EB040008EB040008EB040008EB040008A3
:10018000EB040008EB040008EB040008EB04000893
:10019000EB040008EB040008EB040008EB04000883
:1001A0008D14000800000000D0400B1CD1409C467C
:1001B000203AD34018435242634693401843704755
:1001C0009140031C90409C46203A93401943524270
:1001D0006346D3401943704753B94AB9002908BF51
:1001E00000281CBF4FF0FF314FF0FF3000F07AB90C
:1001F000ADF1080C6DE904CE00F006F8DDF804E07E
:10020000DDE9022304B070472DE9F0478C460D4626
:100210000446089E002B51D18A4217466DD9B2FA86
:1002200082FEBEF1000F0BD0CEF1200C01FA0EF5CC
:1002300020FA0CFC02FA0EF74CEA050C00FA0EF458
:100240004FEA174A250CBCFBFAF81FFA87F90AFB9C
:1002500018CC45EA0C4508FB09F3AB420AD9ED1965
:1002600008F1FF3280F02381AB4240F22081A8F1F7
:1002700002083D44ED1AA4B2B5FBFAF00AFB105592
:1002800044EA054400FB09F9A14509D9E41900F144
:10029000FF3380F00A81A14540F2078102383C44D7
:1002A000A4EB090440EA08400021002E61D024FAA2
:1002B0000EF4002334607360BDE8F0878B4207D9E9
:1002C000002E54D0002186E821000846BDE8F087C2
:1002D000B3FA83F1002940F08E80AB4202D3824210
:1002E00000F2FA80841A65EB03050120AC46002E6B
:1002F0003FD086E81010BDE8F08712B90127B7FBA0
:10030000F2F7B7FA87FEBEF1000F34D1EB1B3A0CBF
:100310001FFA87FC0121B3FBF2F8250C02FB18330E
:1003200045EA03450CFB08F3AB4207D9ED1908F188
:10033000FF3002D2AB4200F2D1808046ED1AA3B268
:10034000B5FBF2F002FB105543EA05440CFB00FC40
:10035000A44507D9E41900F1FF3302D2A44500F205
:10036000B8801846A4EB0C0440EA08409DE73146EB
:100370003046BDE8F087CEF1200405FA0EF307FA07
:100380000EF720FA04F83A0C25FA04F448EA0308B8
:10039000B4FBF2F14FEA184502FB11441FFA87FC47
:1003A00045EA044501FB0CF3AB4200FA0EF409D90F
:1003B000ED1901F1FF3080F08A80AB4240F2878076
:1003C00002393D44EB1A1FFA88F5B3FBF2F002FB49
:1003D000103345EA034500FB0CF3AB4207D9ED1996
:1003E00000F1FF386FD2AB426DD902383D44EB1AB1
:1003F00040EA01418FE7C1F1200722FA07F88B405C
:1004000005FA01F448EA030320FA07FE4FEA134C09
:10041000FD404EEA040EB5FBFCF94FEA1E440CFB0E
:1004200019551FFA83F844EA054509FB08F4AC4264
:1004300002FA01F200FA01FA08D9ED1809F1FF30C9
:1004400043D2AC4241D9A9F102091D442D1B1FFA28
:100450008EFEB5FBFCF00CFB10554EEA054400FB8C
:1004600008F8A04507D9E41800F1FF3529D2A045C6
:1004700027D902381C4440EA0940A4EB0804A0FB39
:1004800002894C45C6464D4615D312D056B1BAEB3B
:100490000E0364EB050404FA07F7CB401F43CC407E
:1004A000376074600021BDE8F0871846F8E6904692
:1004B000E0E6C245EAD2B8EB020E69EB030501386B
:1004C000E4E72846D7E7404691E78146BEE7014684
:1004D00078E702383C4445E7084608E7A8F10208F7
:1004E0003D442BE7704700BF02E000F000F8FEE754
:1004F00072B6394880F30888384880F3098838484C
:100500004EF60851CEF20001086040F20000CCF235
:1005100000004EF63471CEF200010860BFF34F8F39
:10052000BFF36F8F40F20000C0F2F0004EF688512A
:10053000CEF200010860BFF34F8FBFF36F8F4FF013
:100540000000E1EE100A4EF63C71CEF200010860A8
:10055000062080F31488BFF36F8F03F061F903F076
:100560008DF94FF055301F491B4A91423CBF41F86D
:10057000040BFAE71C49194A91423CBF41F8040BAD
:10058000FAE71A491A4A1B4B9A423EBF51F8040B2C
:1005900042F8040BF8E700201749184A91423CBF83
:1005A00041F8040BFAE703F03FF903F0A9F9144C02
:1005B000144DAC4203DA54F8041B8847F9E700F005
:1005C0003FF8114C114DAC4203DA54F8041B884734
:1005D000F9E703F027B9000000090020001100200E
:1005E0000000000800010020000900201844000855
:1005F000001100207411002078110020C82600206E
:10060000A0010008A4010008A4010008A40100083A
:100610002DE9F04F2DED108AC1F80CD0C3689D462E
:10062000BDEC108ABDE8F08F002383F311882846C3
:10063000A047002002F090FE02F0BAFD00DFFEE7C6
:10064000394B6FF007022DE9F0416FF0670100248C
:100650001A7003225A709C70DC701C715C719C7162
:10066000DC711C7259729A72DC7203F045F807460D
:1006700003F092F80546D0BB2C4B9F4239D0013392
:100680009F4239D02A4B27F0FF029A4238D1F8B264
:1006900000F052FAA84642F2107400F07BFC00F021
:1006A00051FA064680B38CBB464635B1214B9F427A
:1006B00003D003F069F800242646002003F026F852
:1006C0004FF090431B6913F0200322D00EB100F0CD
:1006D00033F800F081FC00F015FE00F041FF054604
:1006E000CCB900F0CFFC012002F03CFEF8E78046D8
:1006F000D3E780460446D0E704464FF00108CCE734
:1007000080464FF47A74C8E70446CEE74FF47A7413
:10071000CBE71C46DDE700F023FF401BA042E0D9F9
:1007200000F00AF8D9E700BF78110020010007B0F7
:10073000000008B0263A09B010B51C4B1C4953F80C
:10074000042F013200D110BD8B42F8D1194C1A4B45
:1007500022689A4228D9194B9B6803F1006303F57C
:10076000D0439A4220D202F0E3FF02F0F5FF0020CE
:1007700000F0E2FD124B0220187000F019FE114B40
:10078000DA690022DA61D96999699A619B6972B65E
:100790000D4A0E4B13601B682268202181F31188DB
:1007A0009D4683F30888104710BD00BFFC67000812
:1007B0001C68000804680008FF6700087811002022
:1007C000841100200010024008ED00E000680008DD
:1007D00009490B6849F269009AB21B0C00FB02330D
:1007E000064A0B60136844F2506198B21B0C01FB7F
:1007F0000030106080B270470C11002008110020FA
:1008000010B500211022044600F0ECFD034B03CB91
:10081000206061601868A06010BD00BFACF7FF1FCA
:10082000F0B51F4CBBB000F09BFEA368C31AF92BB8
:1008300030D906AD2346A06028220021284601F0C9
:100840001DFC04F10E0000F0C5FD0023C6B2591DC9
:100850005F1CDBB2B3424FEAC10107DA0E33234417
:100860000822284601F00AFC3B46F0E701230393E7
:100870000823207B02930B4B0193C1F3CF0130235C
:10088000059100930146049503A3D3E9002306488C
:1008900001F0C4F93BB0F0BD78F6339F93CACD8D1B
:1008A000C8210020D5210020A021002070B50D46D0
:1008B00014461E4601F058F950B9022E0ED1012CF3
:1008C0000CD112A3D3E90023C5E90023012070BD98
:1008D000052C14D003D8012C09D0002070BD282C81
:1008E00009D0302CF9D10BA3D3E90023ECE70BA3FB
:1008F000D3E90023E8E70BA3D3E90023E4E70BA344
:10090000D3E90023E0E700BFAFF30080401DA12042
:1009100026812A0B78F6339F93CACD8D9E6AC42117
:10092000818A46EE26417272DF25D7B7F017304A2A
:1009300039059E5638B504460D4603462022284602
:10094000002101F09BFB22792346032A28BF0322C2
:1009500003F8042F28460222202101F08FFB627940
:100960002346072A28BF072203F8052F284603221B
:10097000222101F083FBA2792346072A28BF072200
:1009800003F8062F28460322252101F077FB28468D
:1009900004F108031022282101F070FB382038BD33
:1009A0002DE9F04FADF5017D21AE0EAD40F279128B
:1009B00080460F463046002100F014FD48220021F9
:1009C000284600F00FFD00F0CBFD594B4FF47A7232
:1009D000B0FBF2F0186093E80700012385E80700F8
:1009E0002B740DF15A0000236B74FFF709FF0323EA
:1009F00085F82030F82385F8213007AB18464D499B
:100A000003F0D8F9192228643146284685F83C209D
:100A1000FFF790FF12AB044601460822304601F072
:100A20002DFB0822A1180DF14903304601F026FBE9
:100A30000DF14A03082204F11001304601F01EFBBB
:100A400013AB202204F11801304601F017FB14AB60
:100A5000402204F13801304601F010FB16AB0822A9
:100A600004F17801304601F009FB0DF15903082229
:100A700004F18001304601F001FB04F1880A0DF118
:100A80005A0904F5847B4B465146082230460AF148
:100A9000080A01F0F3FAD34509F10109F3D11BABC0
:100AA00008225946304601F0E9FA04F588744FF0FF
:100AB000000995F834304B4510D84FF0000995F8EF
:100AC0003C304B4515D92B6C21464B44082230460F
:100AD00001F0D4FA083409F10109F0E7AB6B2146C3
:100AE0004B440822304601F0C9FA083409F10109E3
:100AF000DFE7E31DC3F3CF03F97E059300230496DC
:100B00000393BB7E0293193701230093019706A339
:100B1000D3E90023404601F081F80DF5017DBDE8E1
:100B2000F08F00BFAFF300809E6AC421818A46EE39
:100B300088110020F43E0008014B1870704700BF78
:100B400094110020F0B5334B1C7B85B034B1324B8F
:100B50000E221A810024204605B0F0BD2F4A1068ED
:100B6000516802AB03C308230DEB03022C492D4847
:100B700003F0BEF8054630B9274B2B480A221A81EC
:100B800000F0A4FCE6E70169B1F5663F06D9224B07
:100B900026480B221A8100F099FCDCE7438BB3F561
:100BA0007E7F09D01C4A22480C2111814FF47E72AD
:100BB000194600F08BFCCEE71E4A024402F11003F6
:100BC000994204D2144B1C4810221A81E3E71039D1
:100BD0008E1A2046134900F0C7FC3246074605F13D
:100BE0001801204600F0C0FCAB689F4202D1EB68C0
:100BF00098420AD0084B0D221A8100903B46EA68C1
:100C0000A9680E4800F062FCA4E70D4800F05EFC05
:100C10000124A0E7C821002088110020C43D00085D
:100C2000DC97030000680008CC3D0008D83D0008B0
:100C3000EA3D00080898FFF7083E0008253E000836
:100C40004E3E00082DE9F04FADB006AF80460C4691
:100C500000F08AFF054600286AD1237E022B18D1B6
:100C6000E38A012B15D100F07BFC8146FFF7B0FD34
:100C70004FF4C873BD4EB0FBF3F209F5167902FBD1
:100C80001300E37E19FA80F030608BB9B84B002274
:100C90001A709C37BD46BDE8F08F3B1D1D44009582
:100CA000002308224FEAC901204601F04BF84D46C7
:100CB000A38A013BAB425FFA85F90BD905F1010923
:100CC000B9F1110FE9D1AB4BAB4A40F23911AB4846
:100CD00002F0E0FF07F11400FFF792FD2A4607F14A
:100CE0001401381D02F0F4FF03460028CED1B9F1FB
:100CF000100F07D09E4B83F800903368A3F516734E
:100D00003360C6E707F19802014602F8950D2046C8
:100D10000092072201F016F8F9787F2904DD984B3C
:100D2000954A4FF4A871D2E7404600F001FFB0E7C2
:100D3000E38A052B00F0068106D8012BA9D12146B4
:100D40004046FFF72DFEA4E7282B3DD0302BA0D145
:100D5000637E8C4D01336A7BDBB29342E94640F0FF
:100D6000EF80E27E2B7B9A4240F0EA8007F1980305
:100D7000002623F8846D102200933146012320467B
:100D800000F0E0FFB4F81480A8F102081FFA88F818
:100D900008F1030323F003030A3323F00703ADEB49
:100DA000030D0DF1180A33469BB2B11C98454FEA6A
:100DB000C10106F101066CDD5344009308220023B3
:100DC000204600F0BFFFEEE7A38A013B9BB2C92B90
:100DD0003FF65FAF6B4E357B4DBB06F10C030093C6
:100DE00008222B462946204600F0ACFFA38A05F1D5
:100DF0000109013BEDB29D424FEAC90109DA0E3506
:100E00003544009500230822204600F09BFF4D4604
:100E1000ECE700230022C6E900230023B36086F834
:100E2000D730C6F8D830337B0BB9E37E3373002557
:100E300007F114063B1D0822294630467D60BD603F
:100E4000FD6001F01BF93B7A05F10109AB424FEA65
:100E5000C90107D9FB6808222B44304601F00EF97E
:100E60004D46F0E7C1F3CF010023E07E05910496E3
:100E70000393A37E0293193428230146009301941F
:100E800038A3D3E90023404600F0C8FEFFF7C8FCB2
:100E9000FFE695F8D70000F059FAD5F8D8300646A5
:100EA0001BB995F8D70000F061FAD5F8D830434463
:100EB0009E4204D295F8D700013000F057FA4FEA6D
:100EC000980B0024A0B2584504F1010408DA2B68FD
:100ED00080000AEB00010122184400F08BFAF1E7D0
:100EE000D5E90023D5F8D84095F8D70012EB0802D1
:100EF00043F100034444C5E90023C5F8D84000F09D
:100F000025FA844209D395F8D730013385F8D730D4
:100F1000D5F8D8309E1BC5F8D860B8F1FF0F08DCB3
:100F200000232B7300F034FAFFF70CFE08B1FFF733
:100F300003FC2B68144A9B0A013313810023AB6026
:100F4000CD46A6E6BFF34F8F1049114BCA6802F495
:100F5000E0621343CB60BFF34F8F00BFFDE700BFDC
:100F6000AFF3008026417272DF25D7B79C210020A5
:100F700099210020603E0008103F0008B93E00089B
:100F8000DB3E0008C82100208811002000ED00E0B1
:100F90000400FA0508B54FF000530B4A1968914256
:100FA0000AD10A4A597D117009481B7D0373C92271
:100FB00008490E3000F004FAE02200214FF0005002
:100FC000BDE8084000F00EBA9AAD44C59411002067
:100FD000C82100201600002030B5204C20492148AF
:100FE00085B00223637104230025ADF80830012386
:100FF000ADF80C5007228DF80C308DF80B301A4BE1
:101000004B608DF80A2001F023FE184B01950093E8
:101010001749184B18484FF4805200F053FD174BF6
:101020001978254611B1144800F082FD00F098FAB5
:101030000446FFF7CDFB4FF4C87304F51674B0FBFC
:10104000F3F202FB13000E4B14FA80F0186002F06A
:10105000A3FB08B10F232B8105B030BD8811002000
:10106000001100201823002003000600AD0800082E
:1010700098110020450C0008A021002094110020A8
:101080009C2100202DE9F04F94A7D7E900670FF2CB
:101090005429D9E900898D4C93B0DFF850B2DFF8BC
:1010A00050A2204600F006FE0CAD079098B3102227
:1010B0000021284600F096F9079B197B4FF00002AB
:1010C00061F3030219468DF8302051F8040F496886
:1010D0000EAA03C21B680D9A63F31C029DF8303000
:1010E0000D9243F020038DF8303000232A46194634
:1010F000584601F0BDFD079030B9204600F0DEFDF6
:10110000079B8AF80030CCE79AF80030072B3EDCCA
:1011100001338AF8003018220021284600F062F9D5
:10112000DFF8C8A1002319462A46504601F0C8FD41
:10113000014680BB102208A800F054F94FF09042FD
:10114000536983F04003536100F00CFA0B4612A977
:10115000024611E903000DF1240E8EE803009DF80C
:101160003410C1F3030089064CBF0E99BDF8381046
:101170008DF82C0046BFC1F31C0141F00041C1F3C2
:101180000A010891204608A900F0DEFFCAE72046C0
:1011900000F094FDBFE7204600F0E6FC8246002800
:1011A0004AD1DFF850B100F0DBF9DBF800309842AB
:1011B00042D300F0D5F90790FFF70AFB079A8DF8A4
:1011C00020A04FF4C87302F51672B0FBF3F101FBD7
:1011D000130012FA80F0CBF80000DFF81CB19BF886
:1011E000001011B901238DF8203028460791FFF730
:1011F00007FB0799C1F1100A5FFA8AFABAF1060FE4
:1012000028BF4FF0060A524629440DF1210000F094
:10121000D7F80AF10103049308AB03931823029350
:101220002B4B01930123009332463B46204600F0AE
:101230009DFC00238BF8003000F092F9254ADFF87E
:10124000BCA01368C31AB3F57A7F32D3106000F0E4
:1012500089F902460B46204600F036FD204600F094
:1012600083FC30B39AF80C30DFF894B0002B14BF35
:10127000032302238BF8053000F072F94FF47A73E0
:101280002946B0FBF3F0CBF800005846FFF752FBBD
:10129000182307300293104B0193C0F3CF0040F2A4
:1012A000551304900093039542464B46204600F0A8
:1012B0005DFC9AF80C300BB1FFF7B2FA9AF80C30DB
:1012C000002B7FF4EAAE13B0BDE8F08FA021002020
:1012D00098210020A8220020AC220020401DA1203F
:1012E00026812A0BF1C6A7C1D068080F1823002059
:1012F000AD2200209C21002099210020C82100203F
:101300008811002070B502F0E3F8094C094E2070F6
:10131000002530682378834208D902F0D5F8336875
:1013200005440133B5F5D04F3360F2D370BD00BF33
:10133000DC220020B022002002F062B900F100603F
:10134000920000F5D04002F007B90000054B1A6882
:10135000054B1B789B1A834202D9104402F0B4B8A3
:1013600000207047B0220020DC22002038B5074D55
:1013700004462868204402F0ADF828B928682044C3
:10138000BDE8384002F0B8B838BD00BFB022002038
:10139000064991F8243033B100230822086A81F805
:1013A0002430FFF7CBBF0120704700BFB4220020DC
:1013B000022802BF4FF090434FF480029A617047B9
:1013C00010B50023934203D0CC5CC4540133F9E739
:1013D00010BD000002460346981A13F9011B0029AC
:1013E000FAD1704702440346934202D003F8011B2E
:1013F000FAE770472DE9F047234C94F8243005466E
:101400008846174683BB2E46DFF87C90C7B394F816
:1014100024302BB92022FF2148462662FFF7E2FF45
:1014200094F82400C0F10805BD4228BF3D465FFA8C
:1014300085FAAD0041462A4604EB8000FFF7C0FF65
:1014400094F82430A7EB0A079A445FFA8AFABAF1B3
:10145000080F2E44A844FFB284F824A0D6D1FFF789
:1014600097FF0028D2D108E0266A06EB8306B04237
:10147000CAD0FFF78DFF0028C5D10020BDE8F08756
:101480000120BDE8F08700BFB422002070B50C4CED
:101490001C26324600212046FFF7A4FF4823237074
:1014A0000125084B6360657032460021A019FFF7E3
:1014B00099FF49232377044B6577236270BD00BFF2
:1014C000E022002002040048060400480FB4002077
:1014D00004B070470FB44FF0FF3004B07047000005
:1014E000FEE7000000B59BB0EFF309816822684673
:1014F000FFF766FFEFF30583034B9A6B9A6A9A6ACC
:101500009A6A9A6A9B6AFEE700ED00E000B59BB01C
:10151000EFF3098168226846FFF752FFEFF3058376
:10152000044B9A6B9A6A9A6A9A6A9A6A9A6A9B6A4E
:10153000FEE700BF00ED00E000B59BB0EFF30981CE
:1015400068226846FFF73CFFEFF30583034B5A6BB5
:101550009A6A9A6A9A6A9A6A9B6AFEE700ED00E0C4
:1015600002F086B802F060B830B5084D0A449142E6
:101570000BD011F8013B09245840013CF7D040F34F
:1015800000032B4083EA5000F7E730BD2083B8ED1D
:101590000246006848B103681360D388118901339B
:1015A0009BB29942D38038BF1381704770B588B021
:1015B0000D460446202200216846FFF713FF20460F
:1015C0000495FFF7E5FF054658B16B46044608AEA3
:1015D0001A4603CAB24220606160134604F108044F
:1015E000F6D1284608B070BD2DE9F04130B9274B3F
:1015F000274A40F2C531274802F04CFB0B7C23B947
:10160000254B234A40F2C631F5E7C66986B9C16168
:10161000BDE8F081002B29DA930CAB4229D1B4420A
:1016200001D10C60F3E7C8F800100C60BDE8F08150
:101630004B6823F06047BD0C4FEAD37EC3F3807C38
:1016400015EA230538BF3D46B04634466368BEEB15
:10165000D37F23F06042DDD1974203D1C3F380737F
:101660009C450AD1974205E01C46EFE7AA4206D006
:1016700013469D422CBF00230123002BCFD12368AA
:10168000A046002BF0D12160BDE8F081E4410008C4
:10169000D83F00089C420008BD42000808B5034A34
:1016A000034B044840F25E3102F0F4FAB43F000804
:1016B0005C4200089C42000808B503680B60C388C0
:1016C000016033B9044B054A05484FF4C76102F085
:1016D000E1FA013BC38008BD2C4200082840000805
:1016E0009C42000870B50C4600F10C05616831B9E8
:1016F000E38A61F30903E3820020002170BD0E68D4
:101700002846FFF7D9FF6660F0E7000008B5426899
:1017100032B10B4B0B4A0C4840F22F4102F0BAFA9F
:10172000C37DC3F38401013161F38603C375C38AAA
:1017300062F30903C3821B0A62F3C713C37508BDB2
:1017400078420008E43F00089C4200082DE9F04779
:10175000089E32B91F4B204A204840F2395102F00E
:1017600099FA01F007054FEAD6082A4406F0070661
:1017700000EBD1004FF47F49954201D1BDE8F087DD
:1017800005F0070E06F0070AD645774638BF5746DC
:10179000C7F10807511BEC088F4228BF0F46045DB4
:1017A00008EBD60104FA0EF413F801C029FA07FE7B
:1017B00024FA0AF45FFA8EFE8CEA04044EFA0AFE5A
:1017C00004EA0E048CEA040C03F801C03D443E44D4
:1017D000D2E700BFF8410008FC3F00089C42000827
:1017E0002DE9F04106460F4600254FF6FF7441F201
:1017F00021082A4630463946FEF7D6FCC0B284EAB4
:101800000024082314F4004F4FEA4404A4B203F167
:10181000FF3318BF84EA080413F0FF03F2D1083540
:10182000402DE6D12046BDE8F081000010B50A4405
:1018300041F22104914200D110BD11F8013B80EA30
:101840000320082310F4004F4FEA400080B203F158
:10185000FF3318BF604013F0FF03F3D1EAE7000045
:101860002DE9F04F85B08A468DE80C00BDF83C406C
:10187000814630B9494B4A4A40F26E31494802F03C
:1018800009FA11F0604F04D0474B454A40F26F31DE
:10189000F4E7009B002B7ED024B10E9B002B7AD066
:1018A000072C28D809F10C00FFF772FE054628B96D
:1018B0006FF00205284605B0BDE8F08F1422002124
:1018C000FFF790FD22460E9905F10800FFF778FD1D
:1018D000631C2B74009B1B782C4403F01F0363F0E4
:1018E0003F0323724AF000436B6029464846FFF7E6
:1018F0007BFE0125DEE7019B1B0A4FF000080293E7
:1019000000F10C034FF0800B4646454603930398C5
:10191000FFF73EFE07460028CAD014220021FFF739
:1019200061FDB6BB9DF804303B729DF808307B72B8
:1019300002220E9B711E1944B4420AD9B818013212
:10194000D2B211F801EF80F808E00136072AB6B2EA
:10195000F2D1009B197801F01F01B44208BF4FF08B
:10196000400BB81841EA48114BEA010303720132F7
:101970004AF000437B603A7439464846FFF734FE2C
:101980000135B4422DB288F001084FF0000BBED1F2
:1019900090E70022CDE76FF001058BE7E4410008F6
:1019A000C83F00089C420008084200082DE9F047A3
:1019B0001E46CB8A9146C3F30902062A80460F468B
:1019C00019D013460021B0B28DB25A1992B2052A2D
:1019D00009D9A84210D8FA8A034463F30902FA82AB
:1019E0000120BDE8F087A842F3D93A4419F8014034
:1019F00094760131E8E70025FB8A7C68C3F309008F
:101A0000821F1C23B2FBF3FA03FB1A2A1FFA8AF285
:101A10007CB301212368002B39D1B31F03441C2060
:101A2000B3FBF0F301339BB299420CD2BAF1000F31
:101A300009D14046FFF7ACFD08B1C0F800A0206016
:101A400008B304460022B6B24FF0000AB54230D2C5
:101A5000691E49441346E01801339BB211F801EFA7
:101A600080F804E001351C2BADB214D0AE42F2D8A0
:101A7000ECE74046FFF78CFD044608B10023036005
:101A80007C60002CDED16FF00200BDE8F0870131F0
:101A900089B21C46BEE7AE42D8D94046FFF778FD72
:101AA00008B1C0F800A020600028ECD00446002255
:101AB000CCE7FB8AC3F30902164466F30903FB82F1
:101AC0008EE70000F8B50E4615461F46044628B9B5
:101AD000144B154A15484F2102F0DCF8242200214E
:101AE000FFF780FC069B6360079B23626A094FF641
:101AF000FF739A424FF0000028BF1A46A76020707B
:101B0000A061E06197B204F10C05824205D1002387
:101B10002B6027826382A382F8BD2E600130354698
:101B20002036F2E7E0410008543F00089C420008DC
:101B300008B528B9084B094A7321094802F0AAF8E8
:101B4000037823B94BB2002B01DD017008BD054BB2
:101B5000024A7D21F1E700BFE4410008603F000830
:101B60009C42000828410008007870472DE9F7439F
:101B70000D9EBDF828900B9D9DF83040BDF8388033
:101B800007461946104616B9B8F1000F43D11F2C6D
:101B900041D83B78D3B9B8F1070F39D839F00303EE
:101BA00039D1424631464FF6FF70FFF73FFE4FEA0C
:101BB000092920F0010009F44079400449EA04644D
:101BC000400C44EA40244FF6FF730DE043EA09233A
:101BD000B8F1070F43EA0464F5D9FFF701FE424666
:101BE0003146FFF723FE03468DE840012A46214691
:101BF0003846FFF735FE0DB9FFF750FD2B7801335E
:101C0000DBB21F2B88BF00232B7003B0BDE8F0832D
:101C10006FF00300F9E76FF00100F6E72DE9F743F5
:101C20000E9F0B9D9DF83480BDF83C6081469DF869
:101C3000300007B9C6BB1F2836D899F800E0BEF1BE
:101C4000000F34D00C0244F080049DF8281044EAC0
:101C5000C83444EA014444EA0E04072E44EA00640E
:101C600015D919461046FFF7BBFD32463946FFF736
:101C7000DDFD0346019600972A4621464846FFF7B8
:101C8000EFFDB8F1010F0CD125B9FFF707FD4FF6B5
:101C9000FF73EFE72B780133DBB21F2B88BF0023E4
:101CA0002B7003B0BDE8F0836FF00100F9E76FF02F
:101CB0000300F6E7C06900B104307047C1690B68E2
:101CC000C3610C30FFF7F8BC2DE9F84FD0F818A02D
:101CD000DFF86C80054616461F4654464FF0000953
:101CE00000F10C0B0CB9BDE8F88FD4E90223B21A4D
:101CF00067EB0303994508BF90451FD2AB699C422F
:101D0000214628460DD1FFF7EDFCAB691B68AB619E
:101D100021465846FFF7D0FCAC692346A2461C4634
:101D2000E0E7FFF7DFFC2368CAF800302146584699
:101D3000FFF7C2FC5446DAF80030EFE72368EDE71E
:101D400080841E002DE9F04F8BB00D46144607939A
:101D5000DDF850908246002800F06481B9F1000F50
:101D600000F06081531E3F2B00F25C81012A03D1F9
:101D7000079B002B40F05681BAF81460F600002350
:101D8000B5420893099380F053812B199E420AD2E1
:101D9000761B16F0FF0607D1AB4BAC4A40F26751F9
:101DA000AB4801F077FF2646DAF80C3023B9DAF8B1
:101DB0001030002B00F0A5802F2D31D8C5F1300850
:101DC00046454FF000032CBF5FFA88F8B0460093F9
:101DD000294608AB4246DAF80800FFF7B7FCA6EB45
:101DE00008074544FFB2BAF8143003F10053063B2C
:101DF000DB000293DAF80C3005934FF0300B059BB3
:101E0000002B51D087B9DAF81000002861D0002FDC
:101E10005FD0AB4550D98F4B8C4A40F2A651BFE7FB
:101E200037464FF00008DEE7029B23B98A4B874A0A
:101E30004FF4B161B4E7029BE02B28BFE023069387
:101E40005B44AB4204931DD95B1B9F4226BFDBB2B0
:101E500003930397AB4504D97E4B7C4A40F29151E2
:101E60009EE70598CDF8008008ABA5EB0B01039A1F
:101E70000430FFF76BFC039B9844FF1A1D445FFA84
:101E800088F8FFB2049B9B4504D3744B6F4A40F221
:101E90009B5185E7029B069ADDF810B09B1A0293CE
:101EA000059B1B680593AAE7029BBB42ABD26C4B18
:101EB000664A40F2A15173E7CDF800803A46A5EB9F
:101EC0000B0108ABFFF742FCB8443D445FFA88F8C9
:101ED0000027BAF81430B5EBC30F04D9614B5B4A45
:101EE00040F2B1515CE7B8F1400F04D95E4B574A5C
:101EF00040F2B25154E767B15C4B544A40F2B351DF
:101F00004EE70093324608AB2946DAF80800FFF79F
:101F10001DFC731E3F2B35B201D8A64204DD544B85
:101F2000544A40F235213BE760070AD00AAB03EB85
:101F3000D401624211F8083C02F00702134101F893
:101F4000083C082C21D9102C21D9202C8CBF082327
:101F50000423079A002A6DD0B4EBC30F6CD0082C71
:101F600004F1FF3215D89DF8203023FA02F2D10790
:101F700006D54FF0FF3202FA04F423438DF82030E7
:101F80009DF8203089F800304EE00123E1E702237C
:101F9000DFE7102C11D8BDF8203023FA02F2D20767
:101FA00006D54FF0FF3202FA04F42343ADF8203097
:101FB000BDF82030A9F8003036E0202C0ED8089962
:101FC00021FA02F2D30705D54FF0FF3303FA04F4E8
:101FD0000C430894089BC9F8003025E0402C1CD025
:101FE000DDE9086730463946FEF7DEF8002100F0EB
:101FF000010050EA01030BD0224601200021FEF728
:10200000DFF8404261EB410106430F43CDE9086729
:10201000DDE90823C9E9002306E0174B154A4FF410
:102020002071BDE66FF0010528460BB0BDE8F08FCA
:102030001D46F9E7012CA3D0082CA1D9102CB7D943
:10204000202CE5D8C6E700BF344000080C4000084B
:102050009C42000856400008434000087B400008AE
:10206000A3400008CA400008F840000810410008DA
:102070002A4100088C3F00082841000830B585B08F
:1020800030B9244B244A40F2B121244801F002FE29
:1020900023B9234B204A40F2B221F6E7402A04D963
:1020A000204B1D4A40F2B621EFE722B91D4B1A4AD8
:1020B0004FF42F71E9E70024012A0294039417D109
:1020C0001B788DF8083053070AD004AB03EBD2031A
:1020D000554213F8084C05F00705AC4003F8084CCE
:1020E00000910346002102A8FFF730FB05B030BD88
:1020F000082AE5D9102A03D81B88ADF80830E2E792
:10210000202A02D81B680293DDE7D3E90045CDE918
:102110000245D8E764410008A03F00089C4200083F
:102120007F4100082841000870B50C4600F10C05FD
:10213000E16819B9A1602161A18270BD0E682846CD
:10214000FFF7BAFAE660F3E72DE9F04FD1F8009017
:1021500091B0C9F3C01604460D46CDE90223002E06
:1021600050D0C9F3C03BC9F30626B9F1000F80F285
:102170009F8119F0C04F40F09B812B7B002B00F01A
:102180009781BBF1020F03D02278B24240F09381D5
:1021900009F07F02BBF1020F059236D119F07F0FD3
:1021A000C9F30F2A01D10AF0030A2B447606059AD7
:1021B00093F8038046EA0B4646EA82465FEAD81364
:1021C00046EA0A06069300F09A800022002310A92E
:1021D00061E90823059B009367685B4652462046E9
:1021E000B847002800F08880A7698FB9314604F10C
:1021F0000C00FFF7DBF90746D0B96FF0020011B011
:10220000BDE8F08F4FF0020BAFE7C9F3074ACCE708
:102210003B699E420DD03F68002FF9D1314604F151
:102220000C00FFF7C3F907460028E6D0A3693B601E
:10223000A761DDE90801FFF7D3FAB882F97D08F05C
:102240001F06C1F38401711A89B20FFA81FED7E922
:102250000223BEF1000FB8BF01F1200EC9F30461E3
:10226000B8BF0FFA8EFE079152EA030100F02F81EA
:10227000DDE90201801A61EB030102460B469F482B
:102280000021994208BF9042C0F02181069B002B9B
:102290003FD0BEF1010F00F31A8118F0400F38D083
:1022A000DDE90223C7E90223202200210DEB020011
:1022B000FFF798F8DDE90223CDE908232B1D0A93E7
:1022C0002B7BADF836A0013BDBB2ADF834309DF886
:1022D0001C308DF83A309DF814308DF83B30204694
:1022E0008DF838B08DF83960A36808A9984738464A
:1022F000FFF70CFA002082E76FF00B007FE7A76979
:1023000017B96FF00C007AE73B699E4296D03F68A0
:10231000F6E7FB7DC8F34012B2EBD31F40F0CE804E
:10232000C3F38403B34240F0CC8006992B7B4FEA81
:10233000981279B3D2073CD4032B40F2C580DDE973
:102340000223C7E902232B7BAE1D033BDBB23246DF
:10235000394604F10C00FFF729FB002808DA39465A
:102360002046FFF7BFF93846FFF7D0F9032046E7CC
:10237000AB883B832A7B033AD2B2B88A3146FFF757
:1023800055FAFB7DB882DA43C2F3C01262F3C71379
:10239000FB75AFE76AB92E1D013BDBB23246394609
:1023A00004F10C00FFF702FB0028D8DB2A7B013A7E
:1023B000E2E7FA8AC2F30902013B052AD9B250D8F2
:1023C000281D002399420AD907EB020E013210F8AA
:1023D00001CB8EF81AC00133062ADBB2F2D1DDE957
:1023E00002898B4207F11A02CDE908890A9238BFA7
:1023F00004337A680B9234BF5B1900230C93FB8A79
:10240000ADF836A0C3F3090319449DF81C308DF8CC
:102410003A309DF814308DF83B300023ADF834107D
:102420008DF838B08DF839607B602A7BB88A013A24
:10243000291DFFF7FBF93B8BB882834203D1A368C8
:1024400008A92046984708A92046FFF76DFE3846A0
:10245000FFF75CF9B88A3B8B984214BF112000202B
:10246000CDE6786810B34FF0060E03689BB9A2EB77
:102470000E021B2A13D80332024405F1040E1F304A
:102480009942ACD91EF801CB02F801CF013390423A
:10249000DBB2F5D1A3E70EF11C0E1846E5E7184BA9
:1024A000184A194840F2B31101F0F4FB034696E7CD
:1024B0006FF00900A3E66FF00A00A0E66FF00D00D0
:1024C0009DE66FF00E009AE66FF00F0097E6FB7D39
:1024D00068F386036FF3C713FB7539462046FFF791
:1024E00001F9069B002B7FF4D8AEFB7DC3F3840279
:1024F000013262F38603FB7503E700BF80841E0090
:1025000094410008783F00089C4200082DE9F04102
:102510004C4EB04240F081804B4CDFF830E1E56931
:1025200045F00075E561E469846AD4F8007207EA51
:102530000E0747F00107C4F80072D4F8005205EA0C
:102540000E0545F0010545EA0121C4F80012002AF4
:1025500065D00021C4F81C120F46C4F80412C4F858
:102560000C12C4F8141204EBC10501310E29C5F890
:102570004072C5F84472F6D14FF0000E4FF0010CD6
:10258000964510D1826AD2F80032B04223F001039E
:10259000C2F8003253D12C4BDA6922F00072DA61B2
:1025A000DB69BDE8F0819F781D8817F0010F18BF27
:1025B000D4F804820CFA05F11CBF41EA0808C4F8FB
:1025C000048217F0020F1EBFD4F80C8241EA0808FB
:1025D000C4F80C827F0742BFD4F814720F43C4F8CA
:1025E000147204EBC5055F68C5F840729F68C5F8B2
:1025F0004472D4F81C522943C4F81C120C330EF157
:10260000010EBDE7846A0021C4F81C12C4F804124C
:10261000C4F80C12C4F81412AEE7002AF2D1836A8F
:102620000022C3F84022C3F84422C3F80422C3F8AE
:1026300014220122C3F80C22C3F81C22A2E7BDE831
:10264000F08100BF18230020001002400000FFFFAF
:10265000184A916A08B58B688B6013F0010105D0A8
:1026600013F00C0F14BF4FF480310121D80506D5AB
:1026700013F4406F14BF41F4003141F00201D8035C
:1026800006D513F4402F14BF41F4802141F004011A
:10269000D3690BB107489847202383F311880021A1
:1026A000054800F087FE002383F31188BDE8084049
:1026B00001F088B8182300202023002038B5124CE0
:1026C000A36ADD68AA0712D05A6922F002025A6191
:1026D000A36913B1012120469847202383F3118871
:1026E00000210A4800F066FE002383F31188EB0600
:1026F00006D5A36A1021D960236A0BB10248984716
:10270000BDE8384001F05EB81823002028230020DF
:1027100038B5124CA36A1D69AA0712D05A6922F073
:1027200010025A61A36913B1022120469847202361
:1027300083F3118800210A4800F03CFE002383F354
:102740001188EB0606D5A36A10211961236A0BB123
:1027500002489847BDE8384001F034B818230020FB
:102760002823002038B50F4CA36A5D685D602A07F6
:102770000AD5032222701A6822F002021A60636AE4
:1027800013B10021204698476B0706D5A36A9969C3
:10279000236A13B1090403489847BDE8384001F0A3
:1027A00011B800BF1823002010B50F4C204600F0D0
:1027B0003DFA0E4BA3620B21132000F017FA0B21F8
:1027C000142000F013FA0B21152000F00FFA0B2152
:1027D000162000F00BFA002320461A460E21BDE811
:1027E0001040FFF793BE00BF182300200064004094
:1027F0000F4B984210B5044605D10E4BDA6942F0F2
:102800000072DA61DB69A36A01221A60A36A5A685E
:10281000D20707D5626851681268D9611A60064A02
:102820005A6110BD0121082000F07CFCEEE700BFDA
:1028300018230020001002405B87010003291AD8EA
:10284000DFE801F0020A0F14836A9B6813F0E05F6F
:1028500014BF012000207047836A9868C0F380602D
:102860007047836A9868C0F3C0607047836A98684D
:10287000C0F30070704700207047000010B50329B6
:102880001FD8DFE801F0021F2327816A8B68C3F39A
:102890000163183301EB0313107881061ED55468C9
:1028A000C0F30011490041EAC40141F0040100F005
:1028B0000F00586090689860D268DA6041F00101BA
:1028C000196010BD836A03F5C073E5E7836A03F5F9
:1028D000C873E1E7836A03F5D073DDE79488C0F33A
:1028E0000011490041EA4451E1E7000001290CD000
:1028F00003D3022910D000207047836ADA68920758
:1029000001D1186903E001207047836AD86810F08C
:10291000030018BF01207047836AF2E710B539B988
:10292000836AD96889071BD11B699B0704D110BD35
:10293000012915D0022948D1816AD1F8C031D1F8D6
:10294000C401D1F8C8411461D1F8CC4154612024AC
:102950000C610C69A40717D14C6944F0100412E013
:10296000816AD1F8B031D1F8B401D1F8B84114611D
:10297000D1F8BC4154612024CC60CC68A40703D1B9
:102980004C6944F002044C6111795C0864F3041151
:102990009C0864F34511117189064BBF9168118938
:1029A000DB085B0D4CBF63F31C0163F30A01137971
:1029B00048BF916060F3030313714FEA10234FEA9D
:1029C000104058BF11811370508010BD002304497E
:1029D0001A465A50C8180833802B4260F9D1704704
:1029E00044230020026843681143016003B1184783
:1029F00070470000024A136843F0C0031360704739
:102A000000440040024A136843F0C003136070475B
:102A1000004800402DE9F047C66D3768F46934621C
:102A20000546200719D014F0080F0CBF00218021A3
:102A3000E20748BF41F02001A30748BF41F0400131
:102A4000600748BF41F48071202383F31188281D5B
:102A5000FFF7C8FF002383F31188E2050AD520237E
:102A600083F311884FF40071281DFFF7BBFF00238B
:102A700083F311884FF020094FF0000A14F020086A
:102A800031D13B0616D54FF0200905F1380A200652
:102A900010D589F31188504600F04CFA00282FDA3F
:102AA0000821281DFFF79EFF27F0800333600023D5
:102AB00083F3118879060DD562060BD5202383F3A5
:102AC0001188EA6C2B6D9A4201D12B6CF3B900236B
:102AD00083F31188E30621D5AA6E1369F3B1506917
:102AE000BDE8F047184789F31188B38C95F8641056
:102AF0002846194000F0AAFA8AF31188F469BDE764
:102B000080B2308588F31188F469C0E71021281D50
:102B100027F04007FFF766FF3760D8E7BDE8F0878A
:102B200008B50348FFF776FFBDE8084000F04ABE4D
:102B3000C423002008B50348FFF76CFFBDE8084038
:102B400000F040BE3024002037B51D4C1D4D2046FE
:102B500000F070FA009404F11400002320221A49B6
:102B600000F032F92022009404F13800174B184984
:102B700000F0ACF9174BE3652566174C0C212620B5
:102B800000F034F8204600F055FA04F114000094E7
:102B900000232022114900F017F904F138000094B5
:102BA0000F4B1049202200F091F90F4BE3650C21E7
:102BB0002720256603B0BDE8304000F017B800BFFD
:102BC000C4230020005125029C240020F529000880
:102BD000DC2400200044004030240020BC240020DD
:102BE000052A0008FC2400200048004000F1604352
:102BF00000F01F02400903F5614309018000C9B2DA
:102C000000F1604083F8001300F561400123934018
:102C1000C0F880310360704700F16040090100F5A1
:102C20006D40C9B201767047FFF7BEBD00F10802E2
:102C30000123037082600023C26000F11002436030
:102C4000026142618361C3610362436270470000B5
:102C500010B52023044683F31188022303704160DA
:102C6000FFF7C6FD03232370002383F3118810BDF3
:102C70002DE9F0411F4604460D461646202383F3F6
:102C8000118800F108082378042B0ED0294620462D
:102C9000FFF7D4FD48B1204632462946FFF7EEFD46
:102CA000002080F31188BDE8F0813946404600F0ED
:102CB00065FB0028E7D0002383F31188BDE8F0818D
:102CC0002DE9F0411F4604460D461646202383F3A6
:102CD000118800F110082378042B0ED029462046D5
:102CE000FFF704FE48B1204632462946FFF716FE9C
:102CF000002080F31188BDE8F0813946404600F09D
:102D00003DFB0028E7D0002383F31188BDE8F08164
:102D1000F8B5154682680669AA420B46816938BF34
:102D20008568761AB542044607D218462A46FEF749
:102D300047FBA3692B44A3610DE011D93246184625
:102D4000FEF73EFBAF1B3A46E1683044FEF738FB26
:102D5000E2683A44A261A3685B1BA3602846F8BD01
:102D600018462A46FEF72CFBE368E4E783682DE962
:102D7000F041044693421546266938BF856840698C
:102D8000361AB5420F4606D22A46FEF719FB63698A
:102D90002B4463610DE012D93246A5EB0608FEF71D
:102DA0000FFB4246B919E068FEF70AFBE2684244AD
:102DB0006261A3685B1BA3602846BDE8F0812A46D8
:102DC000FEF7FEFAE368E4E710B50A440024C361A5
:102DD000029B006040608460C1608161416102616A
:102DE000036210BD08B582694369934201D18268CC
:102DF00082B98268013282605A1C4261197042694C
:102E000003699A4201D3C3684361002100F0C6FA06
:102E1000002008BD4FF0FF3008BD000070B5202332
:102E200004460E4683F31188A568A5B1A368A2697C
:102E3000013BA360531CA36115782269934224BF10
:102E4000E368A361E3690BB120469847002383F34D
:102E50001188284670BD3146204600F08FFA0028C0
:102E6000E2DA85F3118870BD2DE9F74F05460F466C
:102E700090469A46D0F81C90202686F311884FF091
:102E8000000B144664B1224639462846FFF740FF3E
:102E9000034668B95146284600F070FA0028F1D080
:102EA000002383F31188A8EB040003B0BDE8F08F82
:102EB000B9F1000F03D001902846C847019B8BF35E
:102EC0001188E41A1F4486F31188DBE7C160816131
:102ED0004161C3611144009B0060406082600161F8
:102EE00003627047F8B504460E461746202383F365
:102EF0001188A568A5B1A368013BA36063695A1C4A
:102F000062611E70236962699A4224BFE36863614B
:102F1000E3690BB120469847002080F31188F8BD83
:102F20003946204600F02AFA0028E2DA85F31188B3
:102F3000F8BD0000836942699A4210B501D18268E8
:102F40007AB98268013282605A1C82611C780369F6
:102F50009A4201D3C3688361002100F01FFA204622
:102F600010BD4FF0FF3010BD2DE9F74F05460F465D
:102F700090469A46D0F81C90202686F311884FF090
:102F8000000B144664B1224639462846FFF7EEFE90
:102F9000034668B95146284600F0F0F90028F1D000
:102FA000002383F31188A8EB040003B0BDE8F08F81
:102FB000B9F1000F03D001902846C847019B8BF35D
:102FC0001188E41A1F4486F31188DBE7026843681E
:102FD0001143016003B11847704700001430FFF738
:102FE00043BF00004FF0FF331430FFF73DBF000038
:102FF0003830FFF7B9BF00004FF0FF333830FFF72C
:10300000B3BF00001430FFF709BF00004FF0FF31DD
:103010001430FFF703BF00003830FFF763BF000034
:103020004FF0FF323830FFF75DBF000000207047DF
:10303000FFF78ABD044B0360002343608360C360D5
:1030400001230374704700BFD842000838B5C36934
:1030500004460D461BB904210844FFF7B7FF294673
:1030600004F11400FFF7BEFE002806DA201D4FF41D
:103070008061BDE83840FFF7A9BF38BD024B002290
:103080001B605B609A6070471C250020002303745E
:103090008268054B1B6899689142FBD25A680360AD
:1030A00042601060586070471C25002008B520233E
:1030B00083F31188037C032B05D0042B0DD02BB98F
:1030C00083F3118808BD436900221A604FF0FF3373
:1030D0004361FFF7DBFF0023F2E790E80C001A6082
:1030E00002685360F2E70000002303748268054B16
:1030F0001B6899689142FBD85A680360426010606F
:10310000586070471C250020054B19690874186821
:1031100002681A605360186101230374FDF778BADE
:103120001C25002030B54B1C87B005460A4C10D03A
:1031300023690A4A01A800F059F92846FFF7E4FF7D
:10314000049B13B101A800F06BF92369586907B01B
:1031500030BDFFF7D9FFF8E71C250020AD3000088F
:1031600038B50C4D41612B6981689A6891420446DB
:1031700003D8BDE83840FFF789BF1846FFF786FF40
:1031800001232C61014623742046BDE83840FDF739
:103190003FBA00BF1C250020044B1A681B699068C9
:1031A0009B68984294BF0020012070471C25002096
:1031B00010B5084C236820691A6822605460012207
:1031C00023611A74FFF790FF01462069BDE81040A3
:1031D000FDF71EBA1C25002008B5FFF7DDFF18B16A
:1031E000BDE80840FFF7E4BF08BD0000FEE70000AF
:1031F00010B5174CFFF742FF00F0EAF8802215499E
:10320000204600F06FF8012344F8180C0374124BA9
:10321000124AD96821F4E0610904090C0A431049F3
:10322000DA60CA6842F08072CA600E490A6842F0E9
:1032300001020A601022DA77202283F8222000237C
:1032400083F3118862B60848BDE8104000F06CB8FE
:10325000442500200043000800ED00E00003FA05CB
:10326000F0ED00E0001000E008430008F8B50F4C56
:10327000226A01322262224652F8141F91421546F8
:1032800006D08B68013B8B60202663699A6802B187
:10329000F8BD1968DF68DA604D60616182F31188FA
:1032A0001869B84786F31188EFE700BF1C25002096
:1032B000EFF3118020B9EFF30583202282F3118808
:1032C0007047000010B558B9EFF30584C4F3080443
:1032D00014B180F3118810BDFFF77EFF84F31188CD
:1032E00010BD000082600222027400224274704706
:1032F0008368A3F17C0243F80C2C026943F83C2C50
:10330000426943F8382C074A43F81C2CC26843F83A
:10331000102C022203F8082C002203F8072CA3F13A
:10332000180070472906000810B5202383F3118880
:10333000FFF7DEFF00210446FFF712FF002383F3AF
:103340001188204610BD0000024B1B6958610F20F8
:10335000FFF7DABE1C250020202383F31188FFF736
:10336000F3BF000008B50146202383F3118808202D
:10337000FFF7D8FE002383F3118808BD49B1064B3F
:1033800042681B6918605A60136043600420FFF7AD
:10339000C9BE4FF0FF3070471C25002003689842DB
:1033A00006D01A680260506059611846FFF76EBE79
:1033B0007047000038B504460D462068844200D1AD
:1033C00038BD036823605C604561FFF75FFEF4E78A
:1033D000054B03F114025A619A614FF0FF32DA6132
:1033E00000221A62704700BF1C25002010B5C26081
:1033F0000A4A036153699C68A1420CD85C68036067
:1034000044602060586081609868411A99604FF06C
:10341000FF33D36110BD091B1B68ECE71C2500209E
:10342000036881689A680A449A6042681360036876
:103430005A600023C360024B4FF0FF32DA617047DD
:103440001C25002000207047FEE7000070470000A8
:103450004FF0FF3070470000BFF34F8F024AD36830
:10346000DB07FCD4704700BF0020024008B5074BC3
:103470001B7853B9FFF7F0FF054B1A69120641BFDD
:10348000044A5A6002F188325A6008BDA82600201A
:10349000002002402301674508B5054B1B7833B96E
:1034A000FFF7DAFF034A136943F08003136108BD95
:1034B000A8260020002002407F289ABF00F5803017
:1034C000C0020020704700004FF400607047000009
:1034D000802070477F2808B50BD8FFF7EDFF00F577
:1034E00000630268013204D104308342F9D1012023
:1034F00008BD002008BD00007F2838B5044624D848
:1035000000F0B6F8124D2860FFF7A6FFFFF7AEFFF8
:10351000104BF322DA6002221A612046FFF7CCFF3B
:1035200058611A6942F040021A61FFF795FF4FF4A3
:10353000006100F0FBF8FFF7AFFF00F099F828609A
:103540002046BDE83840FFF7C5BF002038BD00BFAA
:10355000AC260020002002402DE9F84312F00103C0
:10356000144606D0204B40F24B221A600020BDE8E2
:10357000F88385181D4A954204D91B4A4FF41471EB
:103580001160F3E7FFF772FFFFF766FFDFF86C806B
:10359000451A4FF00109012C05EB01060F4604D82E
:1035A000FFF77AFF0120BDE8F883C8F8109031F8E2
:1035B000023B3380FFF750FF0020C8F8100033882B
:1035C0003A889BB29A420DD0074B40F267221A60AC
:1035D000074B1E60074B1C60074B1F60FFF75CFF2B
:1035E000BDE8F883023CD6E7A4260020FFFF0308CD
:1035F00098260020A02600209C26002000200240C3
:10360000084908B50B7828B153B9FFF72FFF0123FC
:103610000B7008BD23B1BDE808400870FFF73CBF40
:1036200008BD00BFA826002038B5FFF741FE0D4BAE
:103630000D4A1C6A11684FF47A7303FB04F38B4242
:103640000A49D1E9004504D2003445F10105C1E938
:103650000045E41845F100051360FFF733FE2046EE
:10366000294638BD1C250020B0260020B8260020A1
:1036700008B5FFF7D9FF4FF47A720023FCF7ACFDD1
:1036800008BD00BF10B50244064B0439D2B29042C7
:1036900000D110BD441C00B253F8200041F8040FC3
:1036A000E0B2F4E750280040104B30B51C6A240407
:1036B00007D41C6A44F440741C621C6A44F400443D
:1036C0001C620B4C236843F4807323600244094B53
:1036D0000439D2B2904200D130BD441C00B251F83E
:1036E000045F43F82050E0B2F4E700BF001002404E
:1036F000007000405028004007B5012201A90020B9
:10370000FFF7C0FF019803B05DF804FB13B5044652
:10371000FFF7F2FFA04206D002A9012241F8044DB2
:103720000020FFF7C1FF02B010BD0000704700008D
:10373000074B45F255521A6002225A6040F6FF725A
:103740009A604CF6CC421A60024B01221A70704704
:1037500000300040C1260020034B1B781BB1034BF7
:103760004AF6AA221A607047C126002000300040A5
:10377000034B1B689B0042BF024B01221A7070472B
:1037800024100240C0260020024B4FF080721A60C5
:10379000704700BF24100240014B1878704700BFEB
:1037A000C0260020064A536823F001035360EFF35C
:1037B0000983683383F30988002383F311887047F2
:1037C00030EF00E010B5202383F31188104B5B68C5
:1037D00013F4006318D0F1EE103AEFF309844FF0C0
:1037E000807344F84C3C0B4BDB6844F8083CA4F174
:1037F000680383F30988FFF7CFFC18B1064B44F840
:10380000503C10BD054BFAE783F3118810BD00BF93
:1038100000ED00E030EF00E0390600083C0600084B
:1038200070470000FEE70000084A094B09498B4237
:1038300004D3094A0021934205D3704752F8040F7C
:1038400043F8040BF3E743F8041BF4E7884400084B
:10385000C8260020C8260020C82600204B684360E8
:103860008B688360CB68C3600B6943614B690362FB
:103870008B6943620B6803607047000008B5194B01
:103880009A6A42F4FC029A629A6A22F4FC029A62F0
:103890009A6A5A6942F4FC025A61134A5B691146FA
:1038A0004FF09040FFF7DAFF104802F11C01FFF7DC
:1038B000D5FF0F4802F13801FFF7D0FF0D4802F1A4
:1038C0005401FFF7CBFF0C4802F17001FFF7C6FF70
:1038D0000A4802F18C01FFF7C1FFBDE8084000F083
:1038E00065B800BF001002402843000800040048EB
:1038F00000080048000C0048001000480014004870
:1039000008B500F08FF9FFF773FCBDE80840FFF73A
:103910002FBF00007047000010B5214CA26A62F46E
:10392000FC02A262A26A02F4FC02A2624FF0FF3122
:10393000A26A226921612269002222612069E0686D
:10394000E160E168E260E168E169164841F08051B8
:10395000E161E169016841F480710160216A01F46B
:103960004071B1F5407F1EBF4FF480332362226265
:10397000236A1B0407D4236A43F440732362236A37
:1039800043F40043236200F02DF9A369064A43F093
:103990000103A361A369136843F02003136010BD02
:1039A0000010024000700040000001401C4B1A68EB
:1039B00042F001021A601A689007FCD55A6822F09A
:1039C00003025A605A6812F00C02FBD1196801F028
:1039D000F90119605A601A6842F480321A601A6854
:1039E0009103FCD50F4A5A604FF40452DA62302238
:1039F0001A631A6842F080721A601A689201FCD544
:103A0000094A122111605A6842F002025A605A684B
:103A100002F00C02082AFAD11A6B1A63704700BF31
:103A2000001002400024050000200240084A08B5AA
:103A3000536911680B4003F00103536123B1054A38
:103A400013680BB150689847BDE80840FFF7BABE4D
:103A50000004014044230020084A08B55369116856
:103A60000B4003F00203536123B1054A93680BB185
:103A7000D0689847BDE80840FFF7A4BE00040140A5
:103A800044230020084A08B5536911680B4003F02D
:103A90000403536123B1054A13690BB15069984778
:103AA000BDE80840FFF78EBE00040140442300201B
:103AB000084A08B5536911680B4003F008035361C5
:103AC00023B1054A93690BB1D0699847BDE8084016
:103AD000FFF778BE0004014044230020084A08B5DF
:103AE000536911680B4003F01003536123B1054A79
:103AF000136A0BB1506A9847BDE80840FFF762BEF1
:103B00000004014044230020174B10B55C691A687B
:103B1000144004F478725A61A30604D5134A936AD8
:103B20000BB1D06A9847600604D5104A136B0BB1ED
:103B3000506B9847210604D50C4A936B0BB1D06BA0
:103B40009847E20504D5094A136C0BB1506C9847AD
:103B5000A30504D5054A936C0BB1D06C9847BDE81A
:103B60001040FFF72FBE00BF000401404423002097
:103B70001A4B10B55C691A68144004F47C425A610F
:103B8000620504D5164A136D0BB1506D9847230595
:103B900004D5134A936D0BB1D06D9847E00404D55A
:103BA0000F4A136E0BB1506E9847A10404D50C4A0E
:103BB000936E0BB1D06E9847620404D5084A136F18
:103BC0000BB1506F9847230404D5054A936F0BB18E
:103BD000D06F9847BDE81040FFF7F4BD00040140E6
:103BE00044230020062108B50846FEF7FFFF062102
:103BF0000720FEF7FBFF06210820FEF7F7FF06214E
:103C00000920FEF7F3FF06210A20FEF7EFFF062149
:103C10001720FEF7EBFF06212820BDE80840FEF73D
:103C2000E5BF000008B5FFF777FEFEF7CFFEFEF711
:103C3000FBFFFFF7FDF9FFF76DFEBDE8084000F060
:103C400001B8000000F00EB808B5202383F31188F6
:103C5000FFF70CFB002383F31188BDE80840FFF752
:103C6000B1BD0000054B064A5A6000229A60072247
:103C70001A6008210B20FEF7CFBF00BF10E000E064
:103C80003F19010008B5062000F078F80120FFF781
:103C9000DBFB00001FB51C46094B1B680546D868B6
:103CA00052B1084B02928DE80A0022462B46064983
:103CB000FDF710FCFFF7E6FF044B1A46F2E700BFE2
:103CC00010110020D0430008DD4300085C3E0008CE
:103CD00010B501390244904201D1002010BD10F806
:103CE000013B11F8014FA342F5D0181B10BD000095
:103CF0002DE9F8430746884691461E468BB10D468E
:103D0000A8EB0500B54207EB000402D20020BDE895
:103D1000F883324649462046FFF7DAFF18B1013DE5
:103D2000EEE7BDE8F8832046BDE8F8831F2938B5E3
:103D300004460D4604D9162303604FF0FF3038BD0A
:103D4000426C12B152F821304BB9204600F030F8E5
:103D50002A4601462046BDE8384000F017B8012B3E
:103D60000AD0591C03D116230360012038BD00245A
:103D700042F8254028469847002038BD024B0146AE
:103D80001868FFF7D3BF00BF1011002038B5074CEB
:103D900000230546084611462360FFF759FB431CE4
:103DA00002D1236803B12B6038BD00BFC4260020B8
:103DB000FFF748BB034611F8012B03F8012B002A3B
:103DC000F9D1704740A2E4F1646891064E6F20611A
:103DD0007070207369670A00426164206677206C06
:103DE000656E6774682025750A0042616420626F01
:103DF0006172645F69642025752073686F756C64F7
:103E00002062652025750A0042616420667720647F
:103E1000657363726970746F72206C656E67746825
:103E20002025750A0042616420617070204352436E
:103E3000203078253038783A30782530387820307E
:103E400078253038783A3078253038780A00476F4E
:103E50006F64206669726D776172650A0000000008
:103E600072656365697665645F756E697175655FB6
:103E700069645F6C656E203C2055415643414E5F3E
:103E800050524F544F434F4C5F44594E414D49435C
:103E90005F4E4F44455F49445F414C4C4F43415452
:103EA000494F4E5F554E495155455F49445F4D411D
:103EB000585F4C454E475448002E2E2F2E2E2F541F
:103EC0006F6F6C732F41505F426F6F746C6F6164E2
:103ED00065722F63616E2E63707000616C6C6F632E
:103EE000617465645F6E6F64655F6964203C3D204A
:103EF000313237006F72672E6172647570696C6F52
:103F0000742E48697465634D6F73616963000000C6
:103F1000766F69642068616E646C655F616C6C6F5C
:103F2000636174696F6E5F726573706F6E7365281D
:103F300043616E617264496E7374616E63652A2CAD
:103F40002043616E61726452785472616E7366656B
:103F5000722A290063616E617264496E697400009F
:103F600063616E6172645365744C6F63616C4E6F14
:103F7000646549440000000063616E6172644861D9
:103F80006E646C6552784672616D650063616E6146
:103F900072644465636F64655363616C61720000B1
:103FA00063616E617264456E636F64655363616CD7
:103FB00061720000696E6372656D656E7454726142
:103FC0006E73666572494400656E717565756554FA
:103FD000784672616D6573007075736854785175B9
:103FE0006575650070726570617265466F724E65C9
:103FF00078745472616E736665720000636F7079D5
:1040000042697441727261790000000064657363F3
:1040100061747465725472616E7366657250617911
:104020006C6F61640000000066726565426C6F63CE
:104030006B0000006269745F6C656E677468203E97
:1040400020300072656D61696E696E675F626974C8
:1040500073203E203000696E7075745F6269745F12
:104060006F6666736574203E3D20626C6F636B5FA4
:104070006269745F6F666673657400626C6F636B10
:104080005F656E645F6269745F6F666673657420F6
:104090003E20626C6F636B5F6269745F6F6666730C
:1040A00065740072656D61696E696E675F626974DF
:1040B0005F6C656E677468203C3D2072656D616958
:1040C0006E696E675F6269747300696E7075745FA4
:1040D0006269745F6F6666736574203C3D2074721C
:1040E000616E736665722D3E7061796C6F61645F9D
:1040F0006C656E202A2038006F75747075745F626D
:1041000069745F6F6666736574203C3D20363400C9
:1041100072656D61696E696E675F6269745F6C6517
:104120006E677468203D3D20300028726573756CA1
:1041300074203E2030292026262028726573756C55
:1041400074203C3D203634292026262028726573B1
:10415000756C74203C3D206269745F6C656E677499
:104160006829000064657374696E6174696F6E20FC
:10417000213D202828766F6964202A29302900767D
:10418000616C756520213D202828766F6964202A9E
:10419000293029006F66667365745F776974686992
:1041A0006E5F626C6F636B203C2028333255202D8C
:1041B000205F5F6275696C74696E5F6F66667365B8
:1041C000746F66202843616E61726442756666652D
:1041D00072426C6F636B2C2064617461292900004A
:1041E0006F75745F696E7320213D202828766F6992
:1041F00064202A29302900007372635F6C656E2089
:104200003E203055000000002863616E5F69642025
:104210002620307831464646464646465529203DBA
:104220003D2063616E5F696400000000616C6C6F2B
:104230006361746F722D3E73746174697374696322
:10424000732E63757272656E745F75736167655FF7
:10425000626C6F636B73203E203000007472616E7D
:10426000736665725F696420213D202828766F6936
:1042700064202A293029000073746174652D3E6220
:1042800075666665725F626C6F636B73203D3D207F
:104290002828766F6964202A293029002E2E2F2E97
:1042A0002E2F6D6F64756C65732F6C696263616E20
:1042B0006172642F63616E6172642E63006974655C
:1042C0006D2D3E6672616D652E646174615F6C6513
:1042D0006E203E203000000000000000F92F000892
:1042E000E52F0008213000080D30000819300008C3
:1042F00005300008F12F0008DD2F00082D300008E0
:104300006D61696E000000002043000860250020F8
:104310009826002001000000ED3100080000000098
:1043200069646C6500000000A0100000000000003F
:10433000FAAAAAAA50040000BFFF000000770000FC
:10434000000000001410AA0000000000AAAAFAAAA7
:1043500004005000FBFF00000000000099770000FF
:104360000000000000000000AAAAAAAA00000000A5
:10437000FFFF00000000000000000000000000003F
:1043800000000000AAAAAAAA00000000FFFF000087
:10439000000000000000000000000000000000001D
:1043A000AAAAAAAA00000000FFFF00000000000067
:1043B000000000000000000000000000AAAAAAAA55
:1043C00000000000FFFF00000000000000000000EF
:1043D0002C2066756E6374696F6E3A20006173738A
:1043E000657274696F6E2022257322206661696C84
:1043F00065643A2066696C6520222573222C206C46
:10440000696E65202564257325730A00FCBDFF7F56
:104410000100000000000000640000000000000037
:10442000FE2A0100D2040000141100200000000048
:10443000000000000000000000000000000000007C
:10444000000000000000000000000000000000006C
:10445000000000000000000000000000000000005C
:10446000000000000000000000000000000000004C
:10447000000000000000000000000000000000003C
:0C44800000000000000000000000000030
:00000001FF
